:100000003F288F00220884002009282084138F08AD
:1000100003193A28F03091000E0880389000F03033
:1000200091030319910003198F0303193A28182823
:100030002B2003010C1820088E1F20088E0803199E
:100040000301900F252880060C28262800000F2881
:10005000841780053A280D080C0403198C0A803097
:100060000C1A8D060C198D068C188D060D0D8C0D35
:100070008D0D3A288313031383126400080083163E
:10008000FF3085000C30860083121E30A8000F3030
:10009000A7000F30AA00912064002408013C031D32
:1000A0006A2886148316861006308312A200103048
:1000B000A00082308E00013001205A308E000230C4
:1000C000012064308E00013001206E308E0002303D
:1000D00001206E288610831686108312640025087E
:1000E000013C031D8C28061483160610063083126B
:1000F000A2001030A0008C308E000130012078303A
:100100008E00023001206E308E00013001206430FC
:100110008E000230012090280610831606108312EC
:100120004B28A601A901A401A5010130AB00640080
:100130002B082802031CA62864000619A028A60A7A
:1001400064008619A428A90AAB0F97286400270821
:100150002602031CAD280130A40064002A082902ED
:0E016000031CB4280130A50008006300B52878
:02400E00F53F7C
:00000001FF
